:100000001EC036C035C034C033C032C0FEC08BC243
:10001000BBC22EC02DC02CC02BC02AC029C028C0F6
:1000200027C026C025C03CC03FC042C02BC02FC047
:1000300030C031C032C034C037C03AC03EC01124D5
:100040001FBECFEDCDBF10E0A0E6B0E0E2EEF5E0E0
:1000500002C005900D92A036B107D9F710E0A0E6D6
:10006000B0E001C01D92A737B107E1F7B6D0B7C223
:10007000C7CF90E0FC013197EC30F10510F5ED5E53
:10008000FF4F09949AD160E270E0BED108958BE2EF
:1000900005C08DE203C086E401C086E631D2089532
:1000A00080E890E0A0D1089580E890E08AD108959A
:1000B00084D160E270E0C6D108957FD160E270E043
:1000C000A3D10895CF92DF92FF920F931F93CF9306
:1000D000DF93182F062FF42EC0D0EC01CC24DD24A2
:1000E0000BC0BBD06C01CC1ADD0A29EBC2162BE089
:1000F000D20610F0802FBDDF2BD1811791F3C601FE
:100100008D5D954025E08B3D920710F48F2DB1DF7A
:10011000C601C39723E0853B920710F4802FA9DF27
:10012000DF91CF911F910F91FF90DF90CF900895B5
:10013000F894A89514BE81B5886181BD11BC1ABA26
:1001400017BA11BA8FEF8BBB88BB82BB8D9A85B76C
:100150008F7A85BF54D09FD091D1F3D078948FEF10
:10016000A1D0C49AC4981BD1A7D00895AFD1882339
:10017000A9F0B3D1863471F0873428F48B3231F092
:100180008D3261F405C0863649F406C089E005C0A9
:100190008AE003C08BE001C08CE06BDFD9D08330F4
:1001A00051F0843018F48130B9F409C0843081F002
:1001B000853091F408C083E061E043E007C081E04E
:1001C00062E044E003C085E065E047E07BDF08953E
:1001D00084E066E048E076DF08951F93A9DF88EBAE
:1001E0009BE044D010E282B3812782BBBFDF85B79A
:1001F000806285BF889585B78F7D85BFF4CF82E00B
:1002000083BF89B7826089BF08951F920F920FB68E
:100210000F9211248F939F938091600090916100C1
:1002200001969093610080936000969902C0C29BF2
:1002300005C0809162008F5F8093620080916200B0
:10024000803221F49698C298109262009F918F910B
:100250000F900FBE0F901F9018958FB7F8942091B4
:100260006000309161008FBFC9010895BC019FB744
:10027000F89440916000509161009FBF8FB7F8944F
:1002800020916000309161008FBF241B350B261731
:100290003707A0F30895BC9AC498BE9ABF9ABD9838
:1002A000C59A08958FB980E48EB98BE101C08DB9EC
:1002B000769BFDCF8FB108951F9310E0C29A84EF13
:1002C00091E0D4DFC2988AEF90E0D0DF969A8AEF6F
:1002D00090E0CCDF96988AEF90E0C8DF1F5F153082
:1002E00069F710E08A9A92988AEF90E0BFDF8A98C7
:1002F000929A8AEF90E0BADF8B9A93988AEF90E017
:10030000B5DF8B98939A8AEF90E0B0DF8C9A94983F
:100310008AEF90E0ABDF8C98949A8AEF90E0A6DFAA
:100320001F5F1530F9F610E0959A8AEF90E09EDF96
:1003300095988AEF90E09ADF1F5F1530A9F71F911B
:1003400008958A98929A8B98939A8C98949A089583
:1003500082990BC0839B09C080B390E024E09695FE
:1003600087952A95E1F7817001C080E0829B04C0E7
:10037000839902C0849982E0829B04C0839B02C05F
:10038000849B83E0829904C0839902C0849984E0AD
:10039000829B04C0839902C0849B85E008958FEFFF
:1003A00093E09BBD8ABD80E48FBD80E882BD83E879
:1003B0008FBD8AE08EBDBB9A08952AB53BB5C901B1
:1003C000089595982AB53BB543E02B3F340728F4B0
:1003D0002AB53BB52C5F3F4F02C02FEF33E03BBD4A
:1003E0002ABD44DF0895959A2AB53BB525303105DD
:1003F00038F02AB53BB5245030403BBD2ABD02C081
:100400001BBC1ABC33DF0895EF92FF920F931F932A
:10041000CF93DF938B019598E82EE7017E01F92EAB
:10042000E70105C0DBBDCABDC80120DF219694E00D
:10043000C030D907B8F3DF91CF911F910F91FF9092
:10044000EF900895EF92FF920F931F93CF93DF9356
:100450008B01959AE82EE7017E01F92EE70105C090
:10046000DBBDCABDC80102DF21972097C9F7DF9124
:10047000CF911F910F91FF90EF9008958E9ABA9AA5
:1004800083E389B912B8549A579A80E090E0FC014E
:10049000EA59FF4F1082019688309105C1F71092FA
:1004A0006300809163008093640080E090E0FC0131
:1004B000E259FF4F1082019688309105C1F71092E2
:1004C00065008091650080937600089580916300B7
:1004D00090916400891B87700895E0916400909169
:1004E000640080916300981731F0809164008F5F01
:1004F000877080936400F0E0EA59FF4F808108958F
:10050000909165009F5F9770209176009217E1F3BC
:10051000539AE0916500F0E0E259FF4F8083909399
:100520006500559A08951F920F920FB60F921124ED
:100530002F938F939F93EF93FF93809163008F5F2F
:10054000877090916400891799F0209165009091CF
:100550007600291769F45E990BC0C29AE091630096
:10056000F0E09CB1EA59FF4F90838093630001C093
:100570008CB15E9AFF91EF919F918F912F910F9087
:100580000FBE0F901F9018951F920F920FB60F92EB
:1005900011248F939F93EF93FF9390917600809116
:1005A0006500981789F0969AE0917600F0E0E2599C
:1005B000FF4F80818CB9809176008F5F8770809328
:1005C00076005E9BFECF02C055985398FF91EF9145
:1005D0009F918F910F900FBE0F901F901895F894D8
:0205E000FFCF4B
:00000001FF
